:1000000000308A00062B0000FF00030E8301A100D0
:100010007F08A0000A08A8008A01A00E0408A20018
:100020007708A3007808A4007908A5007A08A6003C
:100030007B08A700831383128C308400801C222845
:100040008C183528220884002308F7002408F800BB
:100050002508F9002608FA002708FB0028088A006E
:10006000210E8300FF0E7F0E09000130A900BD0A9A
:100070000319BE0ABF0A0319C00A300F40284128DD
:10008000B00A310F44284528B10A2E0F48284928C4
:10009000AE0A2F0F4C284D28AF0A35083604031935
:1000A000552835080319B603B50337083804031972
:1000B0005D2837080319B803B70339083A04031950
:1000C000652839080319BA03B9033B083C0403192E
:1000D0006D283B080319BC03BB0333083404031920
:1000E000752833080319B403B303B2080319792838
:1000F000B2038C108A1122284508F700F70803196B
:1001000086280130770203198A288E28C6018619AD
:10011000C60A8F28C601061BC60A8F28052B2A305F
:100120004507840000084602031DF9292C304507C5
:1001300084000008F700F7080319B328013077029C
:100140000319C328033077020319C328023077024A
:100150000319D028043077020319102905307702DB
:100160000319D429EA29C6080319B728F8292E301B
:10017000450784000008013C0318C2282C304507BD
:100180008400800AF8292E30450784000008283CA6
:100190000318CF282C304507840063308000F829ED
:1001A000C608031DD428F8292E304507840000080E
:1001B000013C03180D292C3045078400800A0130CA
:1001C0004507C70003178E010313470803178D0067
:1001D00083168C130C1483120C08F23C031D0E2999
:1001E0002C30031345078400800A0310450D393E67
:1001F00084008008031D0029840A800803190D2942
:100200000310450D393E8400840A80018403800177
:100210002C30450784006330800003170313F8294E
:100220000310450D353E8400840A8001840380015B
:1002300001304507C70003178E0103134708031752
:100240008D0083168C130C1483120C082A3C03199E
:100250003B29013003134507C90003178E0103131F
:10026000490803178D0083168C130C1483120C0895
:10027000F23C031D9C2903134108033C031D612923
:1002800001304507C70003178E0103134708031702
:100290008D008C0183168C130C15831203130B082D
:1002A000F7008B138316031755308D00AA308D008D
:1002B0008C148C1859290C117708831203138B04A2
:1002C0009A290310450D353E8400840A02308000CF
:1002D0008403583080004108023C031D9A290130F4
:1002E0004507C70003178E010313470803178D0046
:1002F000F2308C0083168C130C15831203130B0839
:10030000F7008B138316031755308D00AA308D002C
:100310008C148C1889290C117708831203138B0411
:100320000310450D353E8400840A023080008403AA
:1003300058308000D02903170313410BA029A429AA
:100340004108023C031DD02901304507C7000317AF
:100350008E010313470803178D002A308C00831683
:100360008C130C15831203130B08F7008B138316E1
:10037000031755308D00AA308D008C148C18BE29BF
:100380000C117708831203138B0442100310450DE0
:10039000353E8400840A0230800084035830800097
:1003A0002C3045078400800A0310450D353E84003B
:1003B000840A0008C80084030008C700C708031D9A
:1003C000E929C808031DE9292C304507840063305A
:1003D0008000F829C6080319F8292E304507840043
:1003E0000008143C0318F8292C30450784008001CC
:1003F000152A2A3045078400460880002E3045071C
:10040000840080012C30450784000008F70001308B
:1004100077020319102A033077020319102A142ACD
:100420002C3045078400800A152A4508F700F70894
:1004300003191F2A013077020319232A272AC6012C
:100440000619C60A272AC601861BC60A272AC60815
:10045000031DE62A0310450D353E8400840A00087A
:10046000C80084030008C700C808031D3B2A4708CA
:10047000053C0318442A0310450D353E8400840AC8
:1004800080018403043080002E3045078400800101
:100490002C3045078400633080000310450D393E41
:1004A0008400840A0008C80084030008C700C70845
:1004B000031D7C2AC808031D7C2A0310450D353E08
:1004C00084008008031D682A840A80080319722AA0
:1004D0000310450D393E8400840A800184030A30EC
:1004E00080007C2A0310450D393E8400840A0330C5
:1004F00080008403843080000310450D393E840061
:10050000840A0008C80084030008C7004808013CAA
:100510000318AE2AFF3A031D912A4708583C0318D6
:10052000AE2A0310450D393E8400840A0008CA0033
:1005300084030008C9004A08033C031CAE2A031DBB
:10054000A52A4908513C031CAE2A0310450D393E2B
:100550008400840A800184030A3080000310450D62
:10056000393E8400840A0008C80084030008C700DC
:100570004808013C031CCB2A031DC22A4708F33C50
:10058000031CCB2A0310450D393E8400840A8001E8
:1005900084030A3080000310450D393E8400840A2C
:1005A0000008C80084030008C700C808031DE52A26
:1005B0004708093C031CE52A0310450D393E840019
:1005C000840A800184030A308000052B0310450D46
:1005D000393E8400840A0008C80084030008C7006C
:1005E0004808013C0318052BFF3A031DFB2A470866
:1005F000583C0318052B0310450D393E8400840A2E
:1006000002308000840358308000003484011F30A1
:100610008305063083169F0060308F000B30F70093
:10062000F71D1C2B073083128101813084000008E4
:10063000C0390F38800083166400813084000008C0
:10064000C03977048000831290011830F800063812
:1006500092009C30831692008C14C03083128B045D
:100660000130B400F430B300BE01BD01C001BF01D0
:10067000B001B101421403081839183C031D7C2B4A
:1006800083160E080239003A0319482B83127C2B7B
:100690008312C4014408013C031C682B2E3044071C
:1006A000840080012C304407840080010310440D35
:1006B000353E8400840A8001840380010310440DC8
:1006C000393E8400840A800184038001C40A4A2BD5
:1006D00003178E0105308D0083168C130C148312C2
:1006E0000C08253C031D792BFA300313B2007B2B39
:1006F00003170313B201D12BC4014408013C031CAE
:10070000B62B2C30440784000008053C031D9C2BAD
:100710000310440D353E8400840A0008C70084039A
:100720000008C6004708023C031C9C2B031D9B2BA2
:100730004608573C0318B42B2E3044078400800130
:100740002C304407840080010310440D353E8400A2
:10075000840A8001840380010310440D393E840023
:10076000840A800184038001C40A7D2B03178E0153
:1007700005308D0083168C130C1483120C08253C55
:10078000031DCF2B03133208323C0318CD2B320844
:10079000F93C031CCD2BFA30B200D12B0317031305
:1007A000B201FF3083168E008312C3010630831618
:1007B0009F0020308500FF3086008113831243089C
:1007C0008500A9080319E12BA9016400061CEA2B86
:1007D000BE01BD01861EEE2BC001BF01C1013E0856
:1007E000003C0318FC2BFF3A031DFA2B3D08F43C98
:1007F0000318FC2B0130C100421C0B2C3E08043CAA
:1008000003180B2CFF3A031D092C3D08DC3C031890
:100810000B2C0230C1004008003C0318182CFF3A92
:10082000031D162C3F08F43C0318182C0330C1009C
:10083000C1080319312C4108023C031D282CB408BF
:10084000031D282C33081D3C031C282CB401B301C4
:10085000B308031D312CB408031D312CB4014630FC
:10086000B300B408031D382C3308323C03183A2C6B
:1008700043123B2C4316C210BE08031D432C3D08F7
:10088000323C0318442CC214C008031D4B2C3F08F3
:10089000323C03184C2CC214C21C552CC319532CC7
:1008A000B4013730B300C315562CC311851E972CE5
:1008B0004108033C031D772C03178E0105308D0082
:1008C0008C0183168C130C15831203130B08F7008D
:1008D0008B138316031755308D00AA308D008C14AE
:1008E0008C18702C0C117708831203138B04410BA6
:1008F000972C03178E0105308D0025308C00831650
:100900008C130C15831203130B08F7008B1383163B
:10091000031755308D00AA308D008C148C188E2C46
:100920000C117708831203138B046430B200B208F1
:100930000319A02C3208313C031CA02C4315A12C18
:100940004311C5017C20350836040319B22C431726
:10095000B308031DB12CB408031DB12CB4016430DD
:10096000B300B32C43130130C5007C203708380492
:100970000319C52CC317B308031DC42CB408031DE9
:10098000C42CB4016430B300C62CC313D62B63004F
:02400E00543F1D
:00000001FF
